:20000000000600205D03000071000000730000000000000000000000000000000000000076
:200020000000000000000000000000007500000000000000000000007700000000000000D4
:20004000A9100000AF100000B5100000BB100000C1100000C7100000CD100000D310000030
:20006000D9100000DF100000E5100000EB100000FEE7FEE7FEE7FEE7FEE70020006880F344
:2000800008887047F048002101724172704710B5ED4B1A7A5C7A511C0907090F8C4201D147
:2000A000012010BDE84C9200403C121990601972002010BDE44E403E34464034217A607A6A
:2000C000814201D130BFF9E7810089198D68002D0CD0401C0007000F6072A8470028EDD083
:2000E00072B62846FFF7D3FF62B6E7E7FFF7CAFFE4E708B5D649D5480860FFF7BEFFD54801
:200100005A2101700026067109210172D24981810A218182D149018308218183CD48022765
:2001200020300776CE498E80CE480880392000020882CD490120088081240C80CA48CB4934
:2001400020300180CA48012180780843C64920310871C849202008760877C6492031087058
:2001600008730874C44881B2C44800F034FB3022C349C44800F01FFBC349012008700C7089
:20018000C1483B210171C0490F200881BE482121017000F027FB00F0F7FABC490620086088
:2001A000AB4980390860BA48012101800321018041210176B74800F0EBF9B74C0020207180
:2001C0000146A148C030417300F091FDB34DE87200F09FFA207A8007FCD5AF49002020318F
:2001E0000870AD490220087207220121002000F0BAF94003010CA948A94B2038818392497B
:200200000446EA7A06464034074640396036C0370094202A53D0602A5CD0A02A7DD000F05F
:200220007EFAA048017D9D4C203C2170017C6170007EA07001209C49E07001C960602046E8
:200240000C22B03000F0B7FA974908221031384600F0B1FA4220608100980D2101730220EC
:20026000B0720F20A87720466026E030067400F03FFE2146A031C87700F04CFE864880214B
:2002800001708A480121017081210170874A952120321180FF218182F100018200210171E1
:2002A0007A49612008606A4980390860208C804930432084A184E97A00293FD041E07D488C
:2002C0008B6748606F487C4981613020F0720020E8752CE0794848606A487949816100200C
:2002E000F0726E4810227749B03000F064FA00984089BE2802D2B87F001DB8775A48203036
:2003000001887322C9B2120289180180564C6E48A08003202081B87F00E00BE002F0DAF90B
:20032000A0814D2020800F2020820020207500F0BAF976E765488B67486072E75C49203173
:20034000A18483216972012189020840603000F0B5F94C485E494160FFF7ACFE082000F042
:2003600025FA3C48403001784906FCD4FFF7C1FE4A4810B52038C08B002802D0002000F019
:200380009DF934482030017F8906890F04D0017F89060AD50A2109E0002101772A48402211
:2003A0006030417B1143417301E00921017726483A4C40380168491C40340160A17B8907AB
:2003C00004D472B64068FFF762FE62B6A07B40070AD51D482030817DC07D814204D072B617
:2003E0003C48FFF754FE62B672B63B48FFF74FFE62B6002010BD70B528494031487A002835
:200400000AD0114E0025254C403E032806D0022808D0012806D04D72002070BD0820E07207
:200420002E4804E002F075FE0420E0722C48706005482022857219482038018C114301849E
:20044000104600F03BF9E7E770010020FF0F000080E100E000300040051D00003B23000084
:2004600000340040010A0000003800401030000060470000006C0040980200200000002018
:200480002814000000010020003C004080E200E000440040201400000060004020000020A9
:2004A0000306000060580040A81400000064004003840000CB1700001B120000B329000069
:2004C00069120000BC2B0000ED020000892C00008B120000371000004D1900003933000060
:2004E0008D310000FA488078032803D0042801D0F8487047F848704770B5F8498A88D2438E
:20050000920707D0F24A2032927F322A02D34009002303E0C200101AC00901233C2801D23C
:200520003C2002E0FF2800D9FF200A8AEC4C120AC01E824215D0002B02D1257B012D03D050
:20054000551DA84200D928460D8A402215430D820D8A4F263540000205430D82088A904359
:200560000882237370BD70B50023DE4D0AE0440064194034A48F260B964207D12405240D2E
:20058000E31840180828F2D3184670BDD64870BDD64A00211170D249012340394B73D449E8
:2005A00003888B8043880B8183888B81C0880882B4201070CB487C30108107209080CB4877
:2005C000022220380272037972B61343037162B6C7482030027AFB231A400272088810221C
:2005E0001043088070470A8810184A88898810180818C04900228A5E8008801A00D500205A
:20060000704770B5022211460020FFF7ACFFB449830828391846FFF7E6FFAD491F22A03198
:200620008A56AB4DAE4C8018A885203C207BAD4E40008019FF3001300383012204211046D4
:20064000FFF791FF4308211D1846FFF7CCFF2886207B032240008019FF3001308384082195
:200660001046FFF780FF0346A11EFFF7BCFFE885207B042240008019FF300130C383082120
:200680000720FFF770FF29464031C880207B022801D3002000E0401C2073914800214038AC
:2006A0004173084670BD944801784222114301709249C014086092490860704730B5844DC6
:2006C000834A2035E97A8F4C4B09D18B0143002B02D0237EDB070AD0938C1940538C1943B9
:2006E000518403D0217FFB231940217700210346D183FE210B40C003C00F0343697A287A1E
:2007000019400843287203D0207FDF210840207730BD7D488121018000210180704700B567
:200720006E48002282806D4940310A747749018077480821818377490183774802707749D8
:20074000812008806C4909200870FFF7E2FF6549734848606B48203001788908890001702B
:200760005B48FF234030C18901339943C1812038C2722038018C2522520111430184A02004
:20078000FFF79CFF002000BD554800216038017341735D4801210180011581800F2101805D
:2007A00002220281018304218182704700E000BF401EFCD27047821801E008C908C09042C7
:2007C000FBD37047821803E00B780370401C491C9042F9D370474118002200E004C0884222
:2007E000FCD370474F48012101704E4A052140321180002202744B4920310A744A4A8A81EE
:2008000013220A700721017270473148C28C110403D5018C4904490C0184418C91430022AC
:200820004184C284002904D13648017F042211430177704726482030017A827A91430022DD
:2008400001728272002904D12E48017F202211430177704710B4214800228088000700D545
:2008600010222B48808B0821C004002800DA0A432E488389DB060CD5042380891A43800635
:2008800007D5134803232030C3762030C3890B43C3810F4B1C24188C01462040504004D0FB
:2008A000A1431143198410BC08E710BC70470C4910B5A0394A7A1E480B2A3DD3094A1D490A
:2008C000116016490A8810239A430A8010BD000000000020085200006450000000340040AD
:2008E0007002002030010020FFFF0000206000400044004020470000003C004080E200E0AE
:2009000000E100E0206C0040004C0040010A0000003000403B3B00000036004000380040DF
:20092000F703000000540040E703000020480040DF2E0000EC0F00008B7A5B1CDCB2FA4B40
:200940008C72012C08D00A2C08D2F849A41E515C0122A2401142B9D11846B7E700238B72D6
:20096000521C4A72B2E70246002002E013785840521C491EFAD270470822012101E00918A1
:200980004008521EFBD2C807C00F7047F0B5E74C00278C3C204626468C3080363D46844625
:2009A000A034607A00280ED1A07A317B884206D20121B940401C0D43A072BF1C34E0002032
:2009C000A07201206072C1B2207A814218D2A07A002819D0092806D26246895C401EC14038
:2009E000C807C00F10E0092805D0FF220120A272491C617208E06046085CFFF7BDFF03E04E
:200A0000607D01214840A175617D012251404840607540000843B8400543A07ABF1C401C2E
:200A2000A072A07D012801D0102FBAD37F1E27757586F0BD70B50546411CBC48401CFFF7BD
:200A400092FFBA49B94C8C394919803188731434ED1C2572207BE07200206072A07260757C
:200A60000226A675FFF792FFB1480188C904617B03D520221143617307E0DF221140617332
:200A800001880122120311430180AA490A8A0C231A430A82A17B00220A2903D2A6498B7FE2
:200AA000322B03D2A4494031C97A00E0C97D8B0601D4FF220132CB0602D401235B021A43FE
:200AC000038803252D02AB4313430380984D9B48203DA8802E810020C043A88100200A06F5
:200AE00000D40820490601D4402108432521084328808E480C38408E2882207D2875FFF72F
:200B000045FFFF200002A88170BD8D494A140B8B002805D093430B83032803D9002207E0DF
:200B200013430B830321484001214003090342187F48018807231B0399431143018070475A
:200B40007A4800B51430417B4908490041733921784809020182818889088900818001887B
:200B6000F022914301800020FFF7CFFF744908208883714880222038018C9143018410464B
:200B8000FFF79CFD00BD6E4A108BC004C10E6A482030007B4000401C1F2800DD1F208142E4
:200BA00000D2481C118B1F231B029943000201431183604908880722120290435E4A4032EB
:200BC000927A5207520D104308807047F8B5574A4109143200290AD0202901DB1F2106E093
:200BE000937B8B4201DA491E01E08B4200DD9173514E4722B77F12020E23B900D3561C3197
:200C00004F4AC918118223377D217843C90000F0CFFB3446A034A17C081A04D4E17C40434C
:200C20004143481100E00020E18A0D18A08AA84200D205463803D22100F0BAFB1F2171563C
:200C4000401908183F49884200D90846F17AA02907D0394920398978032904D0042902D0BC
:200C600004E0394900E039494843000C2082F8BD002130224000C30500D55040491C082948
:200C8000F8D30006000F70472B4910B52031CA8AC0075400C00F04432448CC827430817C53
:200CA000491CC9B281740C2908D32009FFF7E0FF2107090F884201D1012007E6002005E65C
:200CC000014610B522480089224A401C504300F06FFB194980B220314881BE2801D9602072
:200CE000F4E5462801D80020F0E52020EEE5FEB50E4E114C8C3EF01DF930203C009020460E
:200D0000C03035460190C0353046114FE03002903878400605D4608E00281DD130680128D6
:200D20001AD90020FEBD0000E9030000BC010020203800400034004020000020DB050000F0
:200D400000300040FF0F00008020050039050100003C00407017000030680F2870D2029883
:200D6000017B407B8142D3D041008919C0310989401C8C4602070299120F4A73288E401CAE
:200D800080B2288604286FD96046688543002885002251000919C031098A688DCB188142C8
:200DA00001D2698503E0288D814200D92985521C062AEED30199897F491CCAB20199062AE4
:200DC0008A7702D3019A0021917701996046897F49000919C0310882D80805216086C90195
:200DE000401AA12802D30020288691E72B8D688D191A0E2950D9009A00211174C018410814
:200E0000907D61451FD9002811D0907B00280ED0D17D002901D1022807D90020D075012034
:200E2000FFF732FF002828D101E00120D075009900208873C97B491CCAB20099CA7328E06C
:200E400032E0887564E7002806D0D07B002818D0D17D00290BD108E0012090750020D07519
:200E60009074FFF711FF0CE028E0022807D90020D075FFF709FF002803D0602052E7012032
:200E8000D07500990020C873897B491CCAB200998A73052AA9D9D4E70098007C401CC1B24F
:200EA00000982829017403D9608EFFF709FF39E70099002088758873C87329E702280DD0E9
:200EC000002160464A001219C032491C10820629F8D3009900208875087419E76046608635
:200EE000FFF7EEFE45484089C008401E38810FE7424840388078032809D0042807D040495B
:200F000040480289891A0022825E881870473C491531F5E7F8B53C48008B4727C004C40E5B
:200F20003F02B88A0090398B641C411A37480E46604300F03DFA364DC8222880009831463E
:200F4000504300F04BFAFF219131081A6880FE8BF88A311A2F48604300F02AFA80B2A880FF
:200F600015217043614300F023FA192180094901081A00B28D214843C117090E081800129C
:200F8000E880F8BD70B504461F48008B2049C00440394A7DC00E824202D04875FFF7BAFF96
:200FA0001D481B49844203D8022208888A5E1EE019484030844203D3062288888A5E16E0AA
:200FC00015480B88404222188888C01A5043C517AD0E28188011C018062502234D5FCB5E83
:200FE000E91A5143CA17920E51188911CA184443200C801800D5002070BD00004000002027
:20100000310400002047000000300040001A04007002002080920800DA0200001E498A7DB0
:201020000B469200603BD218D064887D401C4007400F8875704730B518480179890628D41F
:20104000174940220A7080220A74134AD47D1546A300603D5B194C330B8304238B82012312
:201060000B720D7972B61D430D71641C6107490FD1750521517562B658210177FF218182C9
:2010800008490182302101710F210170017919430171002030BD000090010020006400406E
:2010A00000600040C6030000B24800680047B14840680047AF4880680047AE48C0680047AB
:2010C000AC4800690047AB4840690047A94880690047A848C0690047A648006A0047A5487C
:2010E000406A0047A348806A0047A248C06A0047F8B5A148027A01790A400272D10719D07D
:2011000001794908490001710021017401709B4C657D9B490223052D09D00E7904252E4344
:201120000E710E8AC127BF00BE430E8265750C791C430C7191070CD50179FD221140017150
:201140008D490020203108708C486038806FFEF79EFFF8BDF8B58A4CA08A218A0840FF216E
:20116000A182864DC62106460E40603D7021495BEA6E02236035002E25D0C4263040002671
:20118000002808D02079184320712020FFF70EFB0620687507E0687D042803D1207B5118B8
:2011A0002039C8776E7501202070032000022082FC2020772671704806700674017949087F
:2011C00049000171F8BD6D4EC707203E768E002F03D0300A20736B75F8BDC006FCD5687DD4
:2011E000022812D021202071FF20C3302082624840230370902303740283891E8182012162
:20120000017202790A430271F8BD267303206875F8BD5C4981200880704710B559493020E1
:201220000876564800224030837D002B0CD00446203C648E0C82047D0C75012B02D0FFF7DD
:20124000A5FB10BD827510BD01230B804E490272897B890602D5807B0428F4D24B48018A2E
:201260000C229143018210BD10B5464C30202076FFF71DFBA08010BD404860380168491CF6
:201280000160434907200872704710B5404C207A800702D53F48FEF7FAFE0720207210BDC6
:2012A00010B53D498B8935488030027B04465200E03C1219C0321381027B521C1207120F97
:2012C00002730F20088310BDF0B5344C0F2020832A490027E031CA8A08461830135CDF2612
:2012E0002F48002B13D08C8A0125A5401D42037802D020252B4300E033400370641CA0B251
:201300008882082802D38F82521CCA82F0BD278002783240027018204874F0BD20497F2098
:2013200088821648E030017C0A060BD41C4A203A127ED20606D5802211430174134A0221DB
:2013400040321174017C09090901891D0174704710B514480178490604D54121017012483C
:20136000FEF795FE11480179C90701D01021017110BD00000001002000600040900100208F
:20138000006400400038004060000020003400400054004071030000004C00400050004019
:2013A000406C0040003C00401F0700004030004030B50B46014600202022012409E00D46AF
:2013C000D5409D4205D31D469540491B2546954040191546521E002DF1DC30BD70B5002411
:2013E0002546002801DA01244042002901DA01254942FFF7DDFFAC4200D04042002C00D015
:20140000494270BD30B47446641E2578641CAB4200D21D46635D5B00E31830BC1847000054
:201420000707070707070707F110000079120000A1120000C912000079000000551100007B
:2014400013120000790000001D1300007900000079000000511300002542313233343536CC
:201460003738393032333435365E4348524953204A454F4E475E393930312A2A3132332AE1
:201480002A2A2A2A3F003B313233343536373839303132333435363D393930313132303015
:2014A00039353133383F0000010058004A616E20333120323031370031303A33303A343364
:2014C00010B5F84801688030826B436C8A1A9A420ADB816383218900818101462031097CBD
:2014E00081730120FFF7A6FA10BD10B5EE48007C00F0E2FA044605281ED8EB49E948621CE1
:2015000010318D30FFF75EF9E6480C2180300173C068E6490840E649884206D1E148006801
:20152000002800D1401EE3498864E2484021203081732046FFF77EFA10BDDA4810B5DE49BE
:2015400080308181D8492039897E81730120FFF771FA10BDD34810B50C21803001731821AB
:201560004173FF2181734021A03081730120FFF761FA10BDF8B5CC4CCE4E8034207E2036B6
:20158000401EC1B22176002917D02746C03FDC20C05B08292AD38A070ED1628BBB8DD21893
:2015A00092B262833B8EC01880B2A083082903D1110961830009A083F8BDB07BC007FBD06B
:2015C000707F0107F8D5C107F6D1810703D5FD2108407077F8BD4107FCD4F72108407077F7
:2015E000B549B448D0314038C185F8BD0629FCD8FFF7C8FC0546608B0B2109074018FFF700
:201600000DFD0521284649070843FFF707FDF88D0D2109074018FFF701FD788E0F21090742
:201620004018FFF7FBFCA5480088000BC10705D04007800F0A21401C484345199A484038A8
:201640008078032818D0042816D0608B152169434843070B00206083A083072138464907E7
:201660000843FFF7DBFC9648818801290DD095498D420CD905200EE0608B15216943484367
:201680009149FFF795FE0746E4E7002003E000880006800F401C60760321C0B289074018FF
:2016A000FFF7BCFC607E41007F48403808186030017C7943CA09112141560A20414388184B
:2016C00000D500207849774DA0310A798035312A1FD0002222764022B2730A46C03A927FA1
:2016E000322A02D3097C4143C8097849884200D90846C0017649FFF75BFE04467148BA3071
:20170000A881AC730120FFF795F9674840388486F8BD012222761022B273727F130705D5FF
:20172000920701D5012602E0022600E0002689797D22D20051430004FFF73AFE65490446D2
:20174000884200D90C466448A881AE73200AE8732C740320D7E7534810B560498030C160BE
:20176000412149020182002181740520FFF762F910BD4C4810B55A49803081814A49403926
:2017800049890A0A12021132C2810174642141745449CA7B82740A7CC274497C0175072024
:2017A000FFF748F910BD404810B54038808DC008FF2800D9FF203B49FF220D3280318A81CC
:2017C00088730120FFF736F910BDF8B5394F787B002802D14448FEF7DBFE364D603D287ABC
:2017E000002820D1E87A2C46603C00281CD0401EE872A07A032816D372B63C48FEF747FC82
:2018000062B6287BE97A401E81427FD120460021803081860186687B800677D427480188C8
:2018200082149143018071E0A07A224E03002036FFF7E8FD0906151A232C2F32676A6C0083
:20184000184800681D2861D90820287315483221803041640120A072FFF7A5FF56E0FFF780
:2018600088FF0220A07251E01E202873FFF773FF0320A0721020B07348E0B07BC00702D0C7
:2018800000F002FB42E000F0C9FA3FE000F01EFE3CE000F062FD39E0B07BC00728D00720C6
:2018A00027E00000300100204000002000FFFFFC0028062C300200200C0500002038004021
:2018C000003400405203000054100000E826000088130000FFFF00000C3100000C510A0090
:2018E0000C71000020470000B01A00003F1C00000520A07200207073B0736948406E386388
:2019000004E000F038FB01E0FFF7DAFD0020F8BD64490822087463483221203841640146A8
:2019200040398A724039096832398163704710B55C48417B0A0703D5F7221140417310BD49
:20194000082211434173FFF7FBF810BDF8B5FEF781FF5348FF224038C4894132214691434E
:2019600002D021461140C1814D494F4D888F0E4660401040803E022700281ED08C87C10538
:2019800007D5E105297801D5394301E0FD2211402970400611D56006308C05D53843308451
:2019A00028780421084304E0B84330842878FB21084028700220FEF781FE3C4804420FD0A9
:2019C0000020210400D50820E10600D53843E10701D004210843334960310A7B02430A7311
:2019E000AE20044225D0200603D501200004FEF765FEA00601D5FEF708FF200711D528496D
:201A00006039C87A202806D0402804D0602806D0802804D005E0C87EFFF77AFF01E000F04C
:201A200042FF600701D5FEF764FBA00701D5FFF77EFF1B484022203004782146914302D046
:201A4000214611400170817F6140114212D084776006308C05D53843308428780421084351
:201A600004E0B84330842878FB21084028700220FEF724FE002C10D0200602D50120FEF7DF
:201A80001DFEA00601D5FEF7D5FE600701D5FEF730FBA00701D5FFF74AFF0020F8BD0000F9
:201AA00080000020D0010020406C0040118000003231320332313214202801D201207047E4
:201AC000802803D220380011801C7047E02803D28038C01008307047E038801014307047D6
:201AE00070B50021C848C943C84DC186288C00041BD4C54C4034E07C401CC0B2E074042852
:201B000001D90420E074C2B2BF49C04838315830FEF758FE207B012108432073298C012042
:201B2000C00301432984FEF7C9FD70BDF8B5B64D06466035A87BB4490090C039C706F00111
:201B400084460846CC1DE031C030F9348E46838EA27C097E002F1EDA490866463143C9B2B9
:201B600076463176002A0AD0072A0AD3FF290BD000290BD055290BD0AA2909D05DE028334C
:201B8000C386521CA27456E0012002E0022000E00420A87351E0009F7F06BF0F4DD0002A94
:201BA00019D0994BC03B1846FF330133F8305B7C092A16D00A2A36D3002E3ED00022A274D0
:201BC000002B23D0E17C8B4224D9891CFEF7CBFE002823D031E0002E2FD13C33C38601202A
:201BE00028E00A21A174185CFEF7C6FEB04224D0607C00281FD0E17C88421CD3A87B400618
:201C000019D5FFF76DFF4C20E07316E00846FFF753FFE074607C401C60740CE0A87B800634
:201C20000BD50820B5E7195C6246490811431954A07C401CA0740020F8BD0120F8BDF8B5ED
:201C4000714D73482C46C03C2646298EFF34A036013481420BD1E88E884207D1E07B002802
:201C600003D0401EE073307B401EF072C9E06748654FA98E403020370090002909D10020B8
:201C80006074A0740F20E886624940200881FEF77BFD8EE041005C4A401CC03A8918C03181
:201CA00000070989000F7873288E401C80B22886032823D8012806D06A8E511889B26986EF
:201CC000032876D106E000206886E073A073A075E0756EE0491C49084C48698641864E4AE8
:201CE00048088018FFF764FB009980B208814749C98A88425DD94549C8825AE04348E030C3
:201D0000C279062093079B0F9840801E52076A8E03D51018884203D320E0101A88421DD9CD
:201D2000E07B401CC0B2E0730A2851D8A07D00280FD0A07B052801D9002005E0022808D976
:201D4000E07D002808D00120FFF7F0FE00283FD1E0750020A0732CE00120F9E7A07B401CDD
:201D6000C0B2A073A17D00290CD0E17D002903D005280CD9012002E00A2808D90020FFF723
:201D8000D5FE25E0E07B022801D90120A075E07B052801D9002005E0022808D9E07D0028DF
:201DA00024D00120FFF7C2FE002811D1E0750020E073397B787B814200D06BE7307B401EF1
:201DC000F072A88E401C80B2A886E98E884218D3FEF79FFC0020C04328860B486030817B43
:201DE0000907090F817303D005203EE70120DDE7A88E317B021D8A4201D2081A35E70420C3
:201E000033E70020F8BD0000F001002000000020FFFF0000003C004000DC050010B5102250
:201E2000FC49FD48FEF7C7FCFA49FB48102220316038FEF7C0FCF8490320D0390865F748F5
:201E40000422017B11430173052260384274F2482021B038C1720F218177F14958200882A9
:201E6000ED48F049503881664166EC48EE494038C185C038016880300164C163436CC91A89
:201E800081634038827210BD70B5E8490888072212029043FF3001300880DF480121703856
:201EA0008172DD4D4020B03DDA49E87210221031D948FEF780FC2C46DD486034A066D948E4
:201EC000D64960660863D5480421C038817220468038818B7D22D2007030D14E91420FD970
:201EE000CC4910223031FEF766FCF82030823720A877D048A0662046CF494030018270BDE7
:201F0000C44910224031FEF756FCFF20713030825520A87770BDC04A0020C049503A096B66
:201F2000526E06E00B4653401B0600D0401C090A120A0B461343F5D17047B84A10B5BF4BA6
:201F4000803A93819073D17310461021A03081730220FEF76FFD10BDB74AB04910B5303AA8
:201F600080398A818873AD482021203081730120FEF760FD10BD70B5A84CA74A2034A07B6F
:201F800002250007000FA073617B1032002902D001290BD03CE0107BC00705D03120FFF749
:201FA000DBFF0120607370BD65730DE00007FBD59A482038017E3129F6D1417E1170817E71
:201FC0005170C07E9070EFE7617B4808CE07491CCBB291496373D039002E0BD0A37BDB0787
:201FE00016D00918964BE0311818FF30097A213001740DE00E18E036317A3679B14205D0F5
:20200000C20700D10420FFF798FF70BD5B1C6373607B0828D8D3411C6173082809D0A07BF0
:20202000C0070BD07D48016B7B4850384166157306E0FFF770FFC1B20020E4E70420107303
:202040007F480521403081720020A07370BDF0B571487038807BC00601D50020F0BD6E48B0
:202060006D491038D039008A898D421A02D50124504201E000241046C10868480023203088
:2020800000290BD0C3758375082202757F2900D97F21002C00D0494248B2F0BD857DAA1858
:2020A00056B28675C27D521CD5B2C575AA07F0D1027D964202DD0121002404E05742BE4244
:2020C00007DA01210C460C2D01D3521C02758375DCE7C375457D6D1CEDB24575202DF6D906
:2020E0004375042AF3D9521EF0E7F0B54A4C5549D03CE08D85B04843000CA087FEF7F2F9C2
:20210000A18D464F48430001010C204640300190018021464A4E603F3446787B8034C031CB
:202120002546C007A0350291002858D00846C038008EFEF727FF019900908880364870386E
:202140000390807BC00747D13348D038408EFEF7D3F90098FEF73AFDB87B042805D233498A
:202160008A88920709D5012206E0042805D92F498A88920701D403228A80FEF7C6FCB97BB1
:202180000A2901D2002008E00F2901D2012004E0142901D2022000E00320244A1288F023D1
:2021A0009A438001024321480280072901D9162100E006211D488181818802888901D208EB
:2021C00018231A4000881143400906221040014303980173FEF7D7FCFFF739FF4DE0FFF761
:2021E00036FF7A7B110748D40B49D0398B8D0299098A8B4205D83168236CC91A124B9942F1
:2022000003DB697F102319436977697FCB061DD437203AE084260000D00000203002002082
:2022200000300040040A0A00DC05000000340040311E1E00311414003C0700000C2000008C
:202240003001002080200500881300008B0714D4080703D57D21FA48C900C185F948818B50
:20226000012319438183052002437A733220606430682838A06305B0F0BD411D0A2902D9A4
:20228000797B090701D5962100E032216164697F0A070AD5021D082A07D88A0702D54908F4
:2022A000490001E0FB2211406977E549E64B40318A6C9C46002A25D033689A1AE34B9A4286
:2022C00001D900228A64E049E04B20398A8D263B9A4207D36246927F2D2A03D2002801DA51
:2022E000002020E003281EDD019AC98A1289914219D10A468F3A082A02D9B839082912D820
:20230000032010E0D04A029B203A1B8AD04F928DDB199A4213D90A7D082A02D33068E06391
:20232000A9E7521C0A75C3218900A181A073614688754020A8730120FEF77CFB9BE700222E
:20234000F0E7BF4810B5C3494038C1601021A03081730120FEF76EFB10BDF8B5B84A1F2303
:20236000203A507BB749C5061B020124002D16DAEF2528405073088B1B2298431202801878
:202380000883B14880222038018C114301841046FEF794F9B048017821430170F8BD45073A
:2023A00011D5FB252840102528435073AB48848002883024A2430280088B09229843120263
:2023C00080180883F8BDA048A030017E002902D0FFF7D0F8F8BD9A49994EC0390C468034B7
:2023E0000B68E16B8E465D1A2E21715E8C46654503DB4821E3630176EAE79149B82640313B
:20240000CD1FF93D7659087B2D680707AD1B002F37D0C60705D0400840000873FFF79AF87A
:20242000F8BD860705D5FD2210400873FFF785F8F8BD460711D5537C002B08D0032B03D266
:2024400081488749203801655B1E537402E0FB2210400873FFF749F8F8BD642D11DA7246FB
:20246000D61A6246B218FF265F36B24209DDF722104008737248062180388172FFF761FFA0
:20248000F8BD606C854203DBA363FFF72EFEF8BD6D482038008EFEF775FD6B492031898821
:2024A000081A00D54042C828F1DD32206064F8BD634810B56B494038C1606021C173102177
:2024C000A03081730220FEF7B5FA10BDF0B55C4C87B06034A07B002205072D0FA573E07B95
:2024E000C10700290DD0002D0BD1617B491CC9B26173032902D2401EE07302E0401CE07333
:2025000062734F4EE77BC03E3046C030E0360590307E0490707E03904B483B00C030C17A1C
:202520000291817A0191417A0091017AFEF76AFF110A0D121420242E353941464E535E633F
:2025400068A4A600FFF7B4FF98E0A80700D5FEE7627393E030200CE004993029F8D1039960
:20256000C17005983849408FA03140BAC885EFE73120FFF7F1FC81E004993129E8D103996E
:202580000170B17E4170F17E8170E1E70079814201D0022024E0072026E0E807D8D0217436
:2025A000D6E740790099814201D0012018E009201AE0E807CCD000986074C9E78079019902
:2025C000814201D004200BE00B200DE0E807BFD00198A074BCE7C0790299814203D00320E5
:2025E000FFF7ABFC4AE00D20E07347E0E807AFD00298E074ACE7FFF78EFCC1B20020EFE795
:202600000F491148EB0740316030002B2CD0096B4166FF210598C331C1850948C03801682B
:2026200080300A46FF3A2D3AC2630164426C891A816303490520803988720F2060771DE014
:20264000F00100200030004020000020DC050000490200000C090000406C00400034004018
:20266000280605000C220000AB0707D5406E08636273E27307B0F0BDFFF7D0FBE07B401C4C
:20268000E073F7E7F304190CEA000D000000000000000000850932047500090000000000B4
:2026A00000000000965A845A963E963D963CA02814000000AA5A965A965A965A965A965A43
:2026C00014000000AA5A965A965A965A965A965A1400000006214843C01C7047F8B500210B
:2026E0000846F94A43009A18C0321289401C51181028F6DB0803010CF44CF54A480861862B
:202700008018FEF755FE274640373881EE484030807A05287ED12046008EFEF733FC2146A1
:20272000B88060310091897BEA4DC907C03400295BD1FEF74BFA2E46803EB07B022808D250
:20274000F98A0905C90E052903D1218AFF3125312182A17F8008081806214843DE49C01CBE
:202760008881DA48408EFDF7C7FEB07B052805D2DA498A88920709D5012206E0052805D9B8
:20278000D6498A88920701D403228A80FEF7BDF9B27B0B2A01D2002108E00F2A01D2012154
:2027A00004E0142A01D2022100E00321CB480388F026B34389010B430380A17E891A00D561
:2027C0000021E27EAB7E4900D21851182183818802888901D20818231A400088114340095E
:2027E00006221040014300980173B848238A878DBB485E1F00210211B7421ADA1C23E35637
:20280000002B0EDB09D0462B0ADD5923DB4323773C2300E03CE0637703E0607F401C207755
:202820001046EB7E012B26D1E976297F491C297721E0268B21779B19BB4216D26177E97E88
:20284000A848002904D10121E976297F491C2977A149898BBB22D200914210D97D22520101
:20286000821A91420BD200230AE097490978CB014B4059B208189849898B9042EAD10C236B
:20288000964A118A0C24A1431943118292498880F8BD10B5FDF7B5FE9348FDF779FEFFF77A
:2028A0001DFF002010BD72B690480179FD22114001718E4962B60020203108708C480121E5
:2028C00001800321018084498A4888807E48082140308172704770B57C4C8749E08D48436D
:2028E000000CA087FDF7FEFDA18D254648430001000C403528800B2000070818FEF78EFB98
:2029000020466030007B032189074018FEF786FBA888052149074018FEF780FBE08D0D21BB
:2029200009074018FEF77AFB608E0F2109074018FEF774FB70BDF0B5704901200880002285
:202940000A816F4B604D1046C4182F18267D80373E73247D0C710C886406FCD4401C092888
:20296000F2D308895849030A80314B75887508462030427282725848594981803021017694
:202980000188102211430180F0BD10B54E495D4888674E480F21203081775B495820088256
:2029A0005148FDF7F5FD594940200881FDF7ECFE10BDF0B5444C85B040342046A77A40308D
:2029C00003904248434AC0300290008A01903F481146808D00903C4820390546A0350668CA
:2029E000687B3B00FEF70EFD06041324E0E09AE0810704D4022108436873FFF7C6FF324860
:202A000000681E2834D9FFF796FF0120CBE00120000386422CD92D484030C08A0005C00EB1
:202A2000052802D102983A4901820398C663B9E0354FC3061DD5EF23184068730520A072DE
:202A40000020C88710773A8B1F2109028A431B210902511839831D488022018C11430184CA
:202A60001046FDF72BFE2B4801780122114301709AE0410710D5FB210840102108436873AD
:202A80001649012088803A8B1F2109028A43092109025118398387E0019A0099914206D231
:202AA00003997D22C96BD200711A914207DBBA8B01231A43BA8305210843687374E00648A4
:202AC0001549818070E00000300100200000002000DC050050020020003800400034004097
:202AE000DF2E00006F170000CC2B00000060004000440040BF5D00008020050000700040B7
:202B0000204700009328000000300040003C0040B6050000406C0040ED020000244F019EFF
:202B2000009BF619B34219D90B7DFA2B03D9214B81261E8001E05B1C0B75029E1C23F356CA
:202B4000002B01D05B1C33771B4B167F9B7E052E06D90026CE87167718330FE00023EBE7FB
:202B6000CE8F4B27761CB6B2FF00CE87BE4208D90026CE871677042B02D91B1F937600E022
:202B80009676C1070CD0E87A401CC0B2E872FA2803D30020E872FFF79EFEFDF7F4FF03E02D
:202BA000000701D40220A072002005B0F0BD0000490200000038004050020020F3041E0831
:202BC00024010900C300123000000E00121112031211120470B5D14C11202070D048CF4910
:202BE000027860310A7140780870CC4D092080352872002008751420FDF7D8FD3120207013
:202C00001420FDF7D3FD712020701420FDF7CEFD0120207120790028FCD1287B4021084319
:202C20002873257C4921A8012818FEF7C1FB06460D2068434921FEF7BBFBB84A203216753C
:202C4000107603202072217B0143217370BD5300D3189B08834206D8904204D85008884244
:202C600001D3052901D20120704700207047AD480068D22806D9AC48017FDF22114001775C
:202C80000020704701207047FEB5A64FA037787B3E46C107603E002919D1400617D50124BF
:202CA000A2487C73818B21438183A1488022018C114301841046FDF701FDB07A042801D166
:202CC0000320B072984820300178214301709948407B002802D19848FDF75AFC944CB07A66
:202CE0002246254660328F494035C03401920300FEF788FB0604202B4E6DFE2A01218F48EF
:202D00008902818088482030017804221143017087480222018C114301841046FDF7CEFC36
:202D200020202072824810228549D030FDF743FD012008E0D07B800701D5032003E008689C
:202D4000262801D90220B072E5E0227E002A19D0607E7C4909280AD300206076521E2276E0
:202D60000879FD221040087119200880D3E0042805D1754A0A800A7902231A430A71401C4F
:202D80006076C8E00320B0720220FDF7BEFEC2E008689628D8D90420B0720020FDF7B5FE10
:202DA000FFF718FF654869490180694981805E4820300178022211430170E889D10108438D
:202DC000E88172B66348FDF762F962B6A3E0E07E002801D0401EE0760878504E800679D1D4
:202DE0005348008EFEF7CEF80090A88050480521008E49074018FEF711F907210098490734
:202E00000843FEF70BF9FDF7BEFE0198807BC0071DD10098FDF7DAFEB87BFDF776FEB87B43
:202E20000F2801D3C02104E0092801D3402100E0002142480288C0231A408A4207D0327BBA
:202E400052085200327302889A430A430280787B0921084201D140207873354F3E49F88DD7
:202E60004843000C0D21B88709074018FEF7D6F8FDF738FBB98D4843218A000B421A207A7F
:202E80005043C217920E10188011081800D5002080B20B21288009074018FEF7BFF8012419
:202EA000347130790028FCD1307C1C498031097AC10079862948FEF77BFA80B20F212881E4
:202EC00009074018FEF7AAF8307BC00702D1307B20433073327C114C4034217A2079FFF754
:202EE000B6FE002801D001203072327C217E00E007E0207DFFF7ABFE00280CD0022030724A
:202F000009E0FFF767FE0420B07204480F2160300175032101740020FEBD000000360040BB
:202F20006047000030010020206C0040003000400000002030020020B01A000000340040AD
:202F4000602F00002038004019300000510A0000030400006F2C00008020050040420F00CE
:202F60004C1D1914E7010D00050000000000000010B5AE480122028081210180AB4B052122
:202F800020331981AA493224497B614395311980232101800F2101838282A6490820086038
:202FA000A5490860A548017840221143017010BDA1490820803108609C49002008809F48C2
:202FC00001789F2211400170704770B59C490126CC8A0A4618328B8AA55C9E40354000D0E4
:202FE0000325002801D0012000E003205B1C9BB268408B82082B05D30023641C8B82A4B202
:20300000CC82A354CC8A0D7DA35CA8400343A354888A401C888270BDF0B5854985B02031C9
:20302000487B8007800F012805D0022809D00020487305B0F0BD8348049020203F270390E1
:2030400005E080482E30049030200F2703907C4C332020766076A076E07620776077A07740
:203060000620E0820720A082002006460190012002900498805D002807D00399411A0198C7
:203080008C464840761C019003E00198844600200290012500950DE06046284206D001200C
:2030A000FFF793FF0098401C009002E00020FFF78CFF6D002F42EFD10098C007C00FFFF7BF
:2030C00084FF02980028D4D102E00020FFF77DFFA08A0728F9D35A48E18A1830085C0006AE
:2030E00001D5CC2000E03320554A193288545449E28A1A315054E28A491C5054E28A491CD7
:203100005054E28A0020491C5054E0820720A0828FE710B54A480021418201744A480122F0
:203120000280812101804849882020310871481546498880464808803020888143482030A9
:203140008283424B40331A81424C8C80384C2034647A022C01D01C7410BD3F4B0B83828108
:20316000828282808A830A210182018301810180FF210231818331487F21818240210172C0
:203180002C49801508602C49086010BD70B5284900232031487A294C02280BD0012809D0CB
:2031A000FFF706FF2449A015803108602372FDF7B6FA39E0224D287C020603D502071CD09F
:2031C000401E2874487B80072ED0688A411C89B26982002816D0082919D07D20C0008142F0
:2031E00000D36B82687C00281ED0401EC0B268740C2811D0002813D016E014484030037410
:203200002B74DFE72078402108432070EAE7FFF703FFFFF7ADFEE5E720782021084302E039
:2032200020789F2108402070002070BD005000404000002080E200E000E100E0406C004032
:2032400070020020581400000038004000340040F30A00000302000005500000F8B55748E1
:203260006421858C203080796843FEF7A1F8544A0123938351490326898C504C7603491E0A
:20328000314380348EB2217A677A8C1C002F04D04F1C874221D9481C24E06B08984201D3E8
:2032A000002005E05D1A181A2F1F874200D23846434F203F3E8394819C1C148202259582A6
:2032C0000D191583851C4E199680C3189B1C1381BD8308180019108013E06D1A2F1F874252
:2032E00000D23846364D203D2E8393839481801C10820223938209181183AB8311809480D2
:203300001081FF2002309083F8BD2E490120088081220A802B4A882120321171284942020F
:2033200020398A80284A0A8000228A81244988832349203108817047F8B520480021203006
:20334000427A224C032A07D021712172202020732074FDF7E4F92FE01D4D194AAF7A0126B6
:20336000203A3B00FEF74EF805041C21281A2700FF22124958328A84322181710F480521F8
:2033800080300172FFF7C1FFFFF768FF08202071092020720A2020730B202074AE720BE0FC
:2033A0000C489080FFF75AFF06E00120400290800320A87200E0A9720020F8BD4000002094
:1833C0002034004000380040F30A0000206C004070010020030200008A
:00000001FF
